:100000002D288001840AFF3E031D01282928A30111
:10001000A200FF30A207031CA307031C29280330FA
:10002000A100DF3015200928A101E83EA000A109A8
:10003000FC30031C1E28A00703181B28A007000083
:10004000A10F1B2820182428A01C282800002828DD
:1000500008008313831203130800FF238316900004
:100060008312073099002030840040300120103086
:100070008500EF308316850001308312A300F43031
:1000800008204428630042288316851283128516AF
:10009000851A4B282F158512851E4F28AF148316FD
:1000A0008516013083122F190301A4000130AF1807
:1000B0000301A40503195F284230AB006628AF1C7A
:1000C00064284330AB0066284130AB0021308316F2
:1000D0009500811304308312A600B030A500712072
:1000E000C9280516AD01A903851977287428851D2F
:1000F0007A287728030105190130A4008518030127
:10010000A40503197428C830072085198828852874
:10011000851D8B288828013005190301A4000301DF
:1001200085180130A4040319852814300720851987
:100130009A289728851D9D289A28030105190130C2
:10014000A40085180301A4050319A7287128F63017
:1001500029020318AD286300AB2808002F12851967
:10016000B228AF28851DB528B2280519B8282F1642
:100170002608A10025081520051264301420051654
:100180002630A100AC30152005126430142005166D
:1001900008000130AA0015302A020318E228851948
:1001A000D228CF28851DD528D22803010519013072
:1001B000A40085180301A4050319DF28E228AA0A70
:1001C000031DCB2842302B020319F2280430A6006D
:1001D000B030A50015302A02031CF2281F30A600FB
:1001E0004030A5002608A8002508A7001F30A6005B
:1001F0004030A500AE2015302A0203180F29030154
:100200002F1A0130A400030185180130A40403193A
:100210000F292808A6002708A5007120C9289030BA
:10022000A5020130031C013EA60226082802031C79
:10023000FA28031D1F2925082702031CFA2828086D
:10024000A6002708A500AE01AE2015302A0203182B
:10025000352903012F1A0130A4000301851801304C
:10026000A404031935297120C928AE0A15302E02BD
:10027000031C2429AE2003012F1A0130A40003011E
:1002800085180130A404031947291430AC00AE20AE
:1002900003012F1A0130A400030185180130A404C2
:1002A00003198129AC0A15302C02031C8029AC03E8
:1002B000AF152F1C60292330A502031CA603642957
:1002C0002330A5070318A60A04302602B03003190C
:1002D0002502031870290430A600B030A5002F10A5
:1002E0001F302602031C8029031D7A294130250274
:1002F000031C80291F30A6004030A5002F14AD0A32
:100300009E2902302C02030103180130A40014308E
:100310002C02013003180301A40503199329AC0131
:100320007120C9289E29AD01AC01AF1D9E29413025
:100330002B0203199E290130AF06AF1106302D02A2
:10034000031CAF29AE2001302F1A0301A400013095
:1003500085180301A4050319A2297120C92847297A
:02036000B029C2
:02400E00443E2E
:00000001FF
